:1000000083018B018A01850186018C019D018F018D
:100010009001910192019301940195019801990138
:100020009A01831610308500003086008117640025
:10003000A73081008312850114309E009F019F0B21
:100040001F289E0B1F2838304B2008304B200130D2
:100050004B200C304B2006304B20C1288316FF303C
:1000600086001830850083120510851405150608D2
:1000700005118039031D2E28851083160030860057
:100080008312080096002E20851005140515160809
:1000900086000511080096002E2085100510051514
:1000A00016088600051108009B010C089C00AA2078
:1000B00003149802031867280314013099020318E7
:1000C0006728031401309A02031867281B149C0345
:1000D0001C08AA2003149902031874280314013081
:1000E0009A02031874281B149C031C08AA200314EA
:1000F0009A0203187D2803147E281B0C00349B01F0
:100100000C089C00AA2003109807031C92280310D7
:1001100001309907031C9228031001309A07031C31
:1001200092281B149C031C08AA2003109907031C87
:100130009F28031001309A07031C9F281B149C035F
:100140001C08AA2003149A07031CA8280314A92832
:100150001B0C00348207003400340A3400340034AD
:10016000643400340334E834003427341034013468
:100170008634A0340F344234403482070D34BB340B
:10018000A03411308C0009308D008E0106309D00A6
:1001900054200318D2288E0A8D03031DC82803306B
:1001A0008C02D5287F2003308C0209308D0010305E
:1001B0001D079B009B031B0884000E088E01800016
:1001C0009D0301300C07031DC82818088F00063056
:1001D0009D00003080384B200F301D078400000840
:1001E00030384220053003151D02031DF9282E303A
:1001F00042209D0BEC280F301D078400000830388A
:100200004220403080384B20203042204D30422068
:10021000483042207A304220003080384B2097010D
:100220008101000000009D010B309E0004309F0002
:10023000EB30A0008B011030850083161F30850045
:1002400083120B1D2629970A0B1129290000000093
:1002500000009E0B21290B309E009F0B21290430AA
:100260009F00A00B2129F8308E000B1D3A29970A18
:100270000B113D290000000000008E0B3529000005
:100280000000000000000301860010308500831686
:100290001730850083120B19970A0B11010899007A
:1002A00017089A009B019B0A851585110B110108FF
:1002B00003111902031953299B0A9B099B0A1B0A64
:1002C0009800103085008316043085008312051DC8
:1002D0006A29C4290030BD20031403111A02031C2B
:1002E0008329031D93290130BD2003110314190232
:1002F000031C8329031D93290230BD200314180217
:10030000031C832993290030BD208F001A08930015
:100310000130BD209000190894000230BD209100EA
:1003200018089500A2290030BD2093001A088F00FC
:100330000130BD209400190890000230BD209500C6
:10034000180891001508031491020318B129031429
:10035000013090020318B129031401308F020318F1
:10036000B1291408031490020318BB2903140130A7
:100370008F020318BB2913088F020F089A00100878
:10038000990011089800E2290230BD200310980757
:10039000031CD429031001309907031CD42903102E
:1003A00001309A07031CD4290130BD20031099079E
:1003B000031CDF29031001309A07031CDF29030106
:0603C000BD209A07C128D0
:00000001FF
